:10C80000251A8D1EDF297C002B7C002DBDC6BD277F
:10C810000A962D913026E2DE01DF250C39CE00018B
:10C820002007CE0001DF1ADE298D7F7EC74DCE00A6
:10C8300040DF29DF1ADE31DF2B398DF28DDFDE2B71
:10C84000DF14DE2EDF03DE27DF2EDF01DE05270506
:10C85000BDC6B3DF27BDC00F250E7C002B7A002D8F
:10C8600026DADE0527010B0C397F0022BDC9A3BDE6
:10C87000C596250E8DA1BDC41F25ED9619B7A0A69E
:10C880009722960084C0972324037AA0E1BDCB09A8
:10C8900025D6D724D023F7A0EB8D0996222715BDE6
:10C8A000C7412029BDC79ACEA0A0FFA0E2C60ED7DF
:10C8B00019D7183996239700BDC4F52562DF20DF0C
:10C8C0001AEE0EDF258DDDFFA0E0BDC74DDE2596FB
:10C8D000239700BDC949254796248D59BDC4F52528
:10C8E0000BBDC60E2620BDC55F240639BDC620255A
:10C8F0002EBDC64CDE01DF27CE0000DF2E8D2125A8
:10C900001EBDC68D25199622261496238D27DE205E
:10C91000FFA0E2BDC7A1BDC6ECBDC794249F0C39E2
:10C9200096238D11BDC7F0250B96248D08BDC83AFE
:10C93000250229EC3997007DA0EB26F8CECBAE7E00
:10C94000C616BDC4F52530EE0EDF01CEA100DF1600
:10C950007FA0A7BDC00C251DB6A0A72605DE08FF39
:10C96000A0AA7CA0A72710BDC6BD26E7D607DE0873
:10C970008D0CFFA0AC861939FEA0E2C610085A261D
:10C98000FC8CA40039CE0000A600436300A1002661
:10C99000086300088C800026EFDF18BDCAD0BDCB2D
:10C9A000030C398DE096181654545454D731108026
:10C9B0000497307F0032398DEA960097249723B789
:10C9C000A0EBCE0006DF27FFA0AEBDC6ECCEA120B7
:10C9D000DF206D0026068DA326F82054FFA0E0EE90
:10C9E0000EDF01FFA0EDDF25BDC8A4BDC73EDE31CF
:10C9F000BDC94E2554CE0000DF2EBDC920254AFEFC
:10CA0000A0E0BDC6FFDE20FFA0E2CEA0A0FFA0E018
:10CA1000C610BDC73EDF20BDC6B3DF27FFA0AEFEF8
:10CA2000A0EDDF01DE31BDC94E251CBDC7A120A68A
:10CA3000DE206F00088CA40026F8DE209627A70EC3
:10CA40009628A70F7EC6AE8620BDC5C620F6FEA0DE
:10CA5000E2C606BDC44A2707BDE1D1085A26F45CE8
:10CA6000BDE0CC5A26FA0C398D098D35BDC794240A
:10CA7000F90C39BDC773BDCB00CECB902057BDC4D8
:10CA8000F524E585F80D26EACE018DDF188DE4CE7C
:10CA9000A120FFA0E26D00273F8D06BDC97826F2D8
:10CAA000398D5D8DA909086D0027FBC6038DB1BDC9
:10CAB000E0CA8D10BDE0CA08088D4B8D49EE00DF3D
:10CAC000017EC3249619A000971924037A0018390F
:10CAD0008D2ECECBB57EE07E8DF6FEA0E2E607275A
:10CAE00012E7008DDFBDE0CAEE0DC60ABDCA608D3B
:10CAF000CE20A8EE0EDF018D0AC608BDCA608DC12A
:10CB00007EC363CE00187EE0C8860136BDC4EA2528
:10CB10002A813A262608A60081332316FFA0E03298
:10CB20008D1A250B36BDC4C8240E306C0020F0864B
:10CB3000123980303125F836BDC4EA3216565656C1
:10CB4000D70039BDC79ABDC4EA2508BDC4F5250480
:10CB500086160D39BDC7A1BDC4F525F7BDC6FFBDFD
:10CB6000C4EABDC7417EC6AE8650BDC59F25E4DE82
:10CB70000D86170827DC096E00BDC42424F9392D61
:10CB80004455502049442052454D4F56453F2004BE
:10CB900046494C45204944202020465420534320F8
:10CBA0004245472E20454E4420204C4F43040D0A59
:10CBB00053574150042A415641494C41424C452A61
:10CBC0002020044C4FC59E434BC9425341C5DB4115
:10CBD00044C6C64F50C7A84E45C71E5245C7D3438B
:10CBE0004FC8695351C9B7414ECA7E4348CB4352DF
:10CBF00055CB68474FCB795349C9854558E0E30089
:0000000000
